:1000000010C01FC01EC01DC01CC01BC01AC019C01C
:1000100018C017C016C015C014C013C012C011C03C
:1000200010C011241FBECFE5D1E0DEBFCDBF20E060
:10003000A0E6B0E001C01D92A936B207E1F783D077
:10004000BFC0DECF813311F4C29A01C0C29880E0F4
:1000500090E00895FC01DA011C9290819623E9F763
:100060008EEF90E00197F1F700C0000082E092E08F
:100070000197F1F700C000008081862319F08C9170
:1000800081608C9382E092E00197F1F700C000005C
:100090008081862319F08C9182608C9382E092E0BB
:1000A0000197F1F700C000008081862319F08C9140
:1000B00084608C9382E092E00197F1F700C0000029
:1000C0008081862319F08C9188608C9382E092E085
:1000D0000197F1F700C000008081862319F08C9110
:1000E00080618C9382E092E00197F1F700C00000FC
:1000F0008081862319F08C9180628C9382E092E05B
:100100000197F1F700C000008081862319F08C91DF
:1001100080648C9382E092E00197F1F700C00000C8
:100120008081682319F08C9180688C9382E092E042
:100130000197F1F700C000008EEF90E00197F1F712
:1001400000C00000089580E886BD16BCD89AD09AF9
:10015000BA9A1092620010926100C3E6D0E040E6C5
:1001600050E062E089E390E075DF8091610090915A
:1001700062009C012F5F3F4F30936200209361002B
:10018000FC01ED59FF4F409160004083263031055E
:1001900021F4109262001092610088818038F9F693
:1001A0008981843AE1F68D818038C9F68A819FEF92
:1001B000980F9230A0F6823091F68B8143DFCFCF3B
:0401C000F894FFCFE1
:00000001FF
